:10000000080C2500D00C02006607040A6606060AE2
:1000100061006607090A01022E00220C8E00030609
:10002000040A1B0C8E000306180A200CE501040AC2
:10003000D70C0200580289019C014306860A7C0005
:10004000690068007E007F007A00BA023F0C06005B
:10005000300C24006A00A3050509A30443062B0AFB
:100060000F0220003F0C84013F0E43063A0AA4020F
:10007000AA022B0A12024306010DFF0FA40432004C
:10008000A40513024306010DFF0F7500A4043300FD
:10009000A4051F02A4043600090C2400860A0802E5
:1000A000E20100080008000800080208030805082B
:1000B00007080A080D08120816081C082208290853
:1000C0003008380841084A0854085F086A0876086A
:1000D000830890089E08AD08BC08CC08DC08ED0831
:1000E000FF08090C2E00400003042F000F032D030E
:1000F0000306CC01EE02750A2C002C032D032C0301
:100100002D032C032D032C032D0300080400FF0CEA
:100110002D002E002F00090C24000B0C3D007F0049
:1001200047040000B50947069C0AD6096606C705BC
:1001300067066B069C0A4605FC0C3F024306AC0AA8
:10014000DF01FD02A80A0306200BBD0200008F0A92
:10015000DF020306F90B8F0A000000000000C7064B
:10016000BF02C704FE03900A260A66070008BF0202
:100170007E004705D60966070008BF0200001C0282
:10018000890138007802A706CE0A4F092900030426
:10019000E70629034704DF03B50A260A000000002A
:1001A00000000000000000000000CA0AC103E80AC5
:1001B00009029C004306040B0306E10ABC0212027A
:1001C000E40AFC001302870521000000000000087B
:1001D000FA02F50A060526051C02000000000000D0
:1001E000000000000000000000081A029C00070642
:1001F000FF0A0000030606040307060500080306BD
:100200002604030726050008870409026706F5028D
:100210000E0B3500D6066704460400086707F50391
:1002200000080B023F0E100D3500D60667050008CA
:10023000100C8400070E4306F80BC706BF02240B00
:10024000090C3D00A4027F004704C704B509470616
:10025000300BD6096606C70567066106300B4604F3
:10026000FC0C3F024306180BDF01FD027A0B03066C
:10027000200B0A028B018C018D018E018F01430737
:10028000E20B6A026B026C026D026E02D609E40098
:10029000080C0600A4050A02EA07680B9801430748
:1002A000610B0B0299014307610B2C0C2400B4076E
:1002B000610B2706610BA3054F0A600B2706860A10
:1002C000740B0A02F00E700F4307860AA305EE0AAC
:1002D00043065D0BB407900143065E0B1A027F0EC6
:1002E0002704430727058A014307610B2B0C2400D1
:1002F000A3054F0A00006003DF02230BFB0B8806F7
:100300001602A20B3E0243068E0B9E008F0B1102BB
:100310003D023F0743060706E706820B96002C00C6
:1003200003042C03180CEC01030C88002D00710948
:10033000090CAD00110203077F0B00000000CD0186
:100340000306160229006B0017024306D40B7F0E2A
:100350002A00F707AE0B040C8800B10B48021F0EF1
:1003600000002E008E076E06C30B2F004306BD0B48
:1003700003042A032B03EE02B90B17027F0E2F0092
:100380000A028F00D40B8A03070ECA012C00070C47
:100390008E002D0071090D022F002C032D032C035C
:1003A0002D03CD008F008A00F707DD0BC90103077D
:1003B00029000000A705A404860A89000306290075
:1003C000DA0B00000000000000000000D609000069
:1003D000000000000000000000000000000000001D
:1003E000860A00000000000000000000000000007D
:0C03F00000000000000000000000E10B15
:10040000840C2700310A800C060A830C2700A00CFC
:10041000C6042900080C2800E6046903C604030684
:10042000C6050000E605E8020C0A0000E60400002C
:10043000C60500000000E605C606E704E604E70777
:10044000470A07020F0EE2012B0A2E0A470A2B0A5F
:10045000310A360A470AA7020A02090AA7020F024E
:10046000090AE605C605A702A10C080AC605000090
:10047000E605080C2800E6050305C60703046F031C
:10048000E604C605E8023B0AE6050000E604C604E9
:10049000E6054A0A4B0AC605E7070008010880037B
:1004A0002F000F03070EE201870AD30B890B910B74
:1004B000550B4D0BF70B0B02F90F43061F0B0002F8
:1004C0002A00A40200022B00A40200022C00F30A5E
:1004D0002400070C4C017E098C07750A6C0620016C
:1004E000FF0F6C0760010402000B400143067B0A0A
:1004F0006C061F0BF70B6C071F0BF70BE2010108D3
:10050000020804080808100820084008800880062F
:10051000C60B0003070EE201AD0BF70BF70BB80B90
:10052000F70BBF0BF70BF70B5F07990AFF06A00A43
:10053000B00A7F079E0A8706A00AB00A8007B00AA1
:100540000706A90A5406AB0A1F0786053F07A6043B
:1005500000085406A40A1F0786043F07A6050008E2
:100560001F0786043F07A604000847046704000F1E
:1005700043063008010F43063108030F43063208D3
:10058000010F43063308070F43063608010F4306E1
:100590003708150F43063808010F43063908030FC3
:1005A00043063A080E0F430634082C0F43063B0857
:1005B000010F43063C08030F43063D08040F4306A2
:1005C0003E08090F43063F086705390F4306050833
:1005D000010F43060D0867044705FF0804020F0ECC
:1005E0000C0F4307340B0B02B5094706F70B6706E0
:1005F0006A07FC0A3500350C4A07680A6A07140BBB
:100600000F0E2A00050900028F014306A3044306CA
:10061000280A00022F00D4060F0BD405F90B03099A
:1006200043060F0BA304280A6706320B0F0E2A009D
:10063000050900028F014307A3044307860AC30686
:10064000230BC305F90B310C2600070C2E006F009D
:100650000400EF03290BEE02270B6600C304A40479
:10066000A304860A80011B0B0A027D0F4306470B79
:10067000010F4306440B0A02070ED501B5094706D0
:10068000F70B6A07140B000B0A02070E410BEB0075
:1006900003046B034B033500F70B8007F70B800354
:1006A000F00EA4043B010F0F5D0B94098006340586
:1006B00000020F0EA4043B01F00F5B013B002F0072
:1006C000A4055B014306680BBF06670546056D0B75
:1006D000DF066D0BBF06670446040F025C0143068C
:1006E000790BFF055F067C0B1F06770BA6058605B9
:1006F0007C0B1F068604FF040F025D014306850B79
:100700003F06A6053F07E705F70B3F06A604E704EB
:10071000F70B1406930BFA06950B0707990B0704C2
:10072000B00B14068B0BFA068D0B0706990B070509
:10073000B00BA70440031E0E2800800608053407EE
:1007400008043407940908024306B60BFD0E43065D
:10075000B00B9406F70BA304870B080C0600660089
:1007600006042604A4047A00BA027C006900F70B90
:10077000740403077405340C20001402000BB40445
:100780000307B405340C20001402000B0C023A00DD
:100790000002120F4306FA04010F4306FA053A0C51
:1007A00024001A02000B00023F0F4307F70BA402BC
:1007B000E006E20B1406E40BFA06E60B0707EA0B69
:1007C0000704B00B1406DC0BFA06DE0B0706EA0B77
:1007D0000705B00B00032F000F031F0E2800400376
:1007E0009F07290034059F06A30BA705F70BD40428
:0807F000C304A304A404860A5B
:0207FE00700C7D
:021FFE00EE0FE4
:00000001FF
